:020000040800F2
:10000000F8290020AD010008732B000861280008C2
:10001000712B0008B1100008F34100080000000037
:10002000000000000000000000000000A52F0008F4
:10003000DD10000800000000DD2C0008ED3D000888
:10004000C7010008C7010008C7010008C701000870
:10005000C7010008C7010008C7010008C701000860
:10006000C7010008C7010008C7010008C701000850
:10007000C7010008C7010008C7010008C701000840
:10008000C7010008C7010008C7010008C701000830
:10009000C7010008C7010008C7010008F5100008E3
:1000A000C7010008C7010008C7010008C701000810
:1000B000C7010008C7010008C7010008C701000800
:1000C000C7010008C7010008C7010008C7010008F0
:1000D000C7010008C7010008C7010008C7010008E0
:1000E000DF100008C7010008C701000800F002F88F
:1000F00000F04DF80AA090E8000C82448344AAF175
:100100000107DA4501D100F042F8AFF2090EBAE872
:100110000F0013F0010F18BFFB1A43F0010318473B
:10012000844B0000A44B0000103A24BF78C878C16B
:10013000FAD8520724BF30C830C144BF04680C60ED
:10014000704700000023002400250026103A28BF35
:1001500078C1FBD8520728BF30C148BF0B60704739
:10016000642900F09F80782900F0D880732900F07E
:10017000E082002070471FB59DE8030000F04AFDB3
:1001800000F03CFB1FBD10B500F0A1FB10BD00F05E
:1001900004FC1146FFF7EFFF04F050F800F008FDF3
:1001A00003B4FFF7F0FF03BC00F0A6FE0948804748
:1001B00009480047FEE7FEE7FEE7FEE7FEE7FEE749
:1001C000FEE7FEE7FEE7FEE704480549054A064B61
:1001D00070470000513E0008ED000008F8230020A1
:1001E000F8290020F8250020F82500200FB4044944
:1001F00010B503AA029800F0A1FA10BC5DF814FB38
:10020000F022002070B5044685690068C10601D55A
:10021000302600E02026C00707D070BDD4E90121B8
:1002200030469047206A401C20626D1EF6D570BD96
:1002300070B5044685690078C00707D170BDD4E960
:10024000012120209047206A401C20626D1EF6D5B7
:1002500070BD70B50C460546012A05D02878800689
:1002600000D5EA69002302E0012305E05B1C93420C
:1002700002D2E05C0028F9D1A869E618C01AA8618A
:10028000286A184428622846FFF7BCFF04E0D5E935
:10029000012114F8010B9047B442F8D32846FFF728
:1002A000C7FF70BD2DE9F04106460024106875298E
:1002B000314616A510D0AFF30080002802DA404284
:1002C00013A507E031688A0701D512A502E04907A6
:1002D00004D511A5012401E0AFF3008000210A221A
:1002E00006F1240709E0B0FBF2FCB0FBF2F302FBDD
:1002F0001C00303078541846491C0028F3D123469E
:100300002A463046BDE8F04100F0A8B900000000E0
:100310002D0000002B0000002000000070B50446F6
:100320000D4621461068AFF300802188090502D5EB
:100330000F4A7A4402E00E4A7A440E32002104F158
:10034000240305E000F00F060009965D5E54491C89
:100350000028F7D120780023000704D5702D02D0A3
:1003600009B1022311322046BDE8704000F076B991
:10037000264900002DE9F05F894604464FF0000A47
:10038000DFF874B1FB44C0F820A02046E16888473C
:10039000002874D0252806D0D4E901219047206A8E
:1003A000401C2062F1E700265F462046E16888474E
:1003B0002028054607DB312D05D2781910F8200CCE
:1003C00008B10643F1E7B00701D526F00406C4F8EA
:1003D0001CA00027C4F818A02A2D09D0284603F035
:1003E00019FF38B304EB8708303DC8F8185019E0FE
:1003F00059F8041B204604EB87029161E1688847A5
:10040000012F054618D1E069002820DA26F02006E1
:100410001DE0D8F8180000EB800005EB40003038F4
:10042000C8F818002046E1688847054603F0F2FE48
:100430000028EED1012F0AD02E2D08D12046E168E8
:1004400088477F1C0546022F46F02006C4DBA069C2
:10045000002803DA404246F00106A061F00701D00F
:1004600026F010066C2D0BD0682D09D04C2D39D0FC
:100470006A2D35D0742D35D07A2D33D016E038E082
:10048000E1682F4620468847B842054609D16C2FBF
:1004900026D04FF48060E168064320468847054631
:1004A00004E06C2F1AD04FF4807006430DB3A5F111
:1004B0004100192802D8203546F400664A462946EC
:1004C000204626604E46FFF74BFE80B101280BD038
:1004D000F61D26F0070000F1080956E74020E4E782
:1004E0008020D8E70020D6E706F104094DE728462A
:1004F00052E7206ABDE8F09FFC48000010B5431C9D
:1005000002E010F8011B71B18107FAD14FF00132FE
:1005100002C88C1A8C4314EAC211F9D0C01A0A0618
:1005200003D0C01E10BDC01A10BD0A0401D0801E29
:1005300010BD0902FCD0401E10BD032A40F23080DD
:1005400010F0030C00F0158011F8013BBCF1020F14
:10055000624498BF11F801CB00F8013B38BF11F895
:10056000013BA2F1040298BF00F801CB38BF00F8AC
:10057000013B11F0030300F0F380083AC0F008805B
:1005800051F8043B083A51F804CBA0E80810F5E70D
:10059000121D5CBF51F8043B40F8043BAFF30080F0
:1005A000D20724BF11F8013B11F801CB48BF11F865
:1005B000012B24BF00F8013B00F801CB48BF00F835
:1005C000012B70474FF000020429C0F0128010F098
:1005D000030C00F01B80CCF1040CBCF1020F18BF1F
:1005E00000F8012BA8BF20F8022BA1EB0C0100F0B2
:1005F0000DB85FEAC17C24BF00F8012B00F8012B85
:1006000048BF00F8012B70474FF0000200B51346B9
:1006100094469646203922BFA0E80C50A0E80C5022
:10062000B1F12001BFF4F7AF090728BFA0E80C50D3
:1006300048BF0CC05DF804EB890028BF40F8042BCC
:1006400008BF704748BF20F8022B11F0804F18BF39
:1006500000F8012B70477047704770472DE9F0474D
:100660000D4699469246044600F124080168880622
:1006700004D5E06921F01001216000E00120A842CA
:1006800001DD471B00E00027A1697A1902EB090090
:10069000081AA0612078C00602D42046FFF7B2FDF8
:1006A000002608E0D4E901211AF806009047206AE4
:1006B000401C761C20624E45F4DB2078C0060AD52B
:1006C0002046FFF79FFD06E0D4E901213020904746
:1006D000206A401C2062381EA7F10107F4DC07E005
:1006E000D4E9012118F805009047206A401C2062D7
:1006F000281EA5F10105F3DC2046FFF799FD2078BF
:10070000000602D50220BDE8F0870120FBE710B506
:10071000436913B1AFF3008001E0FFF79AFD0120B8
:1007200010BD127800F124010A7000224A700122E3
:10073000EDE711684FF0FF32E9E70000074B70B5B5
:100740000D467B4400F043F80446284600F052F87A
:1007500010B14FF0FF3070BD204670BDDF3A000091
:1007600010B5203AC0F00B80B1E81850203AA0E84C
:100770001850B1E81850A0E81850BFF4F5AF5FEA80
:10078000027C24BFB1E81850A0E8185044BF18C933
:1007900018C0BDE810405FEA827C24BF51F8043BDA
:1007A00040F8043B08BF7047D20728BF31F8023B2E
:1007B00048BF11F8012B28BF20F8023B48BF00F8C2
:1007C000012B704701694A1C02610878704700B527
:1007D0008FB0CDE901310021059105497944CDE97A
:1007E000031011466846FFF7C5FD0FB000BD0000BD
:1007F000E5FFFFFF007B00F08000704710B5424826
:100800005421FFF701FF41485421FFF7FDFE404806
:100810005421FFF7F9FE3F493B483C4A3F4B0860F3
:100820003D490A603A491960531C0365481C10652C
:10083000012008653B48344A39A1784400F01CF98E
:1008400020B9384878440A3800F0BBF937482F4AB5
:1008500035A1784400F010F920B9344878440A38BA
:1008600000F0AFF932482A4A2FA1784400F004F989
:1008700020B92F4878440A3800F0A3F940232248D1
:10088000DC000021224600F0D4F820B1254878444D
:10089000543800F096F91D4822464023002100F00C
:1008A000C8F820B121487844543800F08AF9184833
:1008B00022461023002100F0BCF8002806D01C4876
:1008C0007844BDE81040563800F07BB910BD1048A0
:1008D00070B5006D20F001040B4800F043F90B489F
:1008E00000F040F90A4800F03DF909E0206D20F0E1
:1008F0000105204600F036F9204600F073F82C463A
:10090000002CF3D170BD00009C220020F0220020BA
:1009100044230020500000205400002058000020F4
:1009200072000000574400007700000043440000BC
:100930002F4400000EB5CDE90001FFF7DFFD029066
:1009400069460120ABBE0EBD08B569460090022085
:10095000ABBE08BD1FB58DE8070069460520ABBEDC
:1009600004B010BD1FB58DE80F0069460620ABBE70
:10097000F6E708B5694600900920ABBE08BD1CB576
:10098000CDE9000169460A20ABBE1CBD704708B521
:10099000694600900C20ABBE08BD754600F018F902
:1009A000AE4605006946534620F00700854618B05C
:1009B00020B5FFF709FCBDE820404FF000064FF0DE
:1009C00000074FF000084FF0000B21F00701AC4684
:1009D000ACE8C009ACE8C009ACE8C009ACE8C009A3
:1009E0008D46704770B50446051F00F0F7F80068A3
:1009F000002C14BF446870BD002C18BFAC423CBF33
:100A000020466468F8D301680A18AA4218BF4560F6
:100A100003D12A6805461144016028684119A142A2
:100A20001CBF6C6070BD6168696021680844286003
:100A300070BD70B5C468A50713D0650211D4B2F5B6
:100A4000807F09D0B2F5007F06D0B2F5806F08D163
:100A5000012300F1240106E05D1E6FF07F46B542E0
:100A600001D3012070BD0161C361416024F4706154
:100A70001143C160002070BD2DE9F0410C460746CE
:100A80001646104600F06EF82078611C61280AD0E6
:100A9000722802D077283CD102E00125002405E02D
:100AA0000225042402E0082448F2020511F8010B93
:100AB0002B2806D0622809D011F8010C74280AD01E
:100AC0000BE045F0030544F00204EFE745F00405B0
:100AD00044F00104EAE744F0100438462146FFF7E9
:100AE00029FF411C15D00021316171604FF4007164
:100AF000F560F1617061200704D5304602220021C3
:100B000000F0E6F8306D40F0010030653046BDE899
:100B1000F0810020FBE72DE9F0410D460646104C20
:100B2000206DC10704D0410804D020F00104F7E78C
:100B300022460EE0542000F09CF807000ED0206DF5
:100B400047F001010843542120653846FFF75CFD5A
:100B50003A4629463046BDE8F0418DE70020D6E709
:100B60009C2200202DE9F04704464FF000094FF089
:100B7000FF37C568D4E90486A80707D0204600F0EF
:100B800057F93046FFF7E0FE002802DA3846BDE8A4
:100B9000F087280502D54046FFF724FF4C21204668
:100BA000FFF732FD206D20F0010020654846EEE79A
:100BB00010B50446AFF300802046BDE81040FFF7B3
:100BC000EFBA10B500F07EF9BDE8104000F074B93E
:100BD0000048704798230020704700000048704785
:100BE000A0230020704770477047704738B504460F
:100BF0000A4600206946AFF30080002808BF38BDD0
:100C000002460099204600F084F9012038BD0120F9
:100C100000F0D3B9F8B5AFF30080054600200C46CC
:100C2000102000BF0646A819A0420DD932466946D9
:100C30000020AFF30080070008BF00F0BEF9009865
:100C4000A04218BF0546C419FFF7C8FF0560074654
:100C5000F01D20F007004619284600F053F9B44271
:100C600008BFF8BDA21B31463868BDE8F84000F067
:100C700050B970B50646FFF7B1FF056806F10B00E5
:100C800020F00704B4429CBF002070BD2B466A6868
:100C9000BAB11068A04210D304F1080188423CBFE9
:100CA0005068586007D35168101941601168091BDA
:100CB000016058601460101D70BD13465268002A10
:100CC000E7D121462846FFF791FF0028DED170BD0D
:100CD0002DE9F041044616460D464769007B800722
:100CE0002ED03846FFF745FE50BB3EB3012E02D052
:100CF000022E25D104E0204600F025F905441DE030
:100D00003846FFF744FEE168002841F01001E16039
:100D100005DA204600F058F80120BDE8F081C9034B
:100D20000BD56268E16A914200D81146A26911446C
:100D30002269891A814200DD08460544002D01DA46
:100D40000220EAE7E16A6068E268814206D2910324
:100D5000E06203D522F4003141F01002A6690027B9
:100D6000AE4213DCE16A814201D90B4600E0034642
:100D700003EB060C2369ACEB030CAC4506DD8142AA
:100D800001D98C4600E084469C4505D1A7602760C8
:100D900042F02000A5620DE0AD1BE669AE1B81426A
:100DA000A66000D90846C01A281A20605819606049
:100DB00022F0200003490840E060002084F84870D9
:100DC000ABE70000BFCFD7FFC16821F4001141F0AD
:100DD0008001C16000218160016070472DE9F0470A
:100DE000814614460E464FF0FF383248D5685769A1
:100DF000054209D03846A169FFF7C1FD002811DB83
:100E00002C48C0430540E5602B46324649463846EB
:100E1000FFF7A0FDA16920F00042B21A114400289A
:100E2000A16103D02046FFF7CFFF4046BDE8F08721
:100E300070B504460569C06A6168884200D80846F2
:100E4000E16821F42011E160C90312D5A84208D05D
:100E50002246411B2846FFF7C1FF10B14FF0FF307B
:100E600070BD0020E562C4E90150E06820F48030E4
:100E7000E060002070BD10B50446C06820F020007E
:100E8000E060A16AA06988420DD02046FFF7D0FF3C
:100E9000E06820F4405040F01000E060A06AA061DB
:100EA0002069E062606044F24001E0688843E060ED
:100EB00010BD000010000200002801D000F01CB896
:100EC0007047000010B5014602A000F05DF8012057
:100ED00010BD000053494752545245443A205265D0
:100EE0006469726563743A2063616E2774206F7061
:100EF000656E3A200000000001491820ABBEFEE7F5
:100F00002600020000210160C0E901107047102096
:100F10007047034640688C46002818BF88423CBF93
:100F200003464068F8D318681844884207D00CF18B
:100F3000030020F00700001D411A521A0146081D47
:100F40000A60FFF74FBD10B50146C268900703D095
:100F5000900607D5886A0AE000F03EF8012101609A
:100F6000881E10BD8B69486818440B69C01A91F837
:100F700048301BB191F84910401A10BD1103FCD53F
:100F80000028FADD401E10BD70B505460C460A204B
:100F900000E06D1C00F018F835B128780028F8D171
:100FA00002E0641C00F010F814B120780028F8D199
:100FB000BDE870400A2000F007B810B500F010F846
:100FC000BDE81040FFF778BF08B569468DF800000E
:100FD0000320ABBE08BD00000048704798230020E6
:100FE00010B5012805D0002103A0FFF7CDFF012097
:100FF00010BD09A1F8E7000053494752544D454D33
:101000003A204F7574206F662068656170206D65A9
:101010006D6F7279000000003A2048656170206DA4
:10102000656D6F727920636F72727570746564009C
:1010300008B100207047014870470000740000208C
:1010400032B1054B03EB401040F8212000207047DF
:101050006FF00100704700007C22002010B54FF0B7
:10106000FF3430B9FFF7E4FF18B123B101F07AF88B
:1010700004E0204610BD142300F040FE0028F9D003
:10108000012010BD38B54FF0FF34049D30B9FFF793
:10109000CFFF18B125B100F0DDFF05E0204638BDD7
:1010A0001424009400F0DDFE0028F8D0012038BDA3
:1010B000FEE730B590F840500124AC40C56B6C6041
:1010C000046863604368102B036803D0996000686C
:1010D000C26030BD9A600068C16030BD704710B515
:1010E0004FF48054204600F0B3F82046BDE810408D
:1010F00000F0AAB810B5202000F0AAF8402000F0B7
:10110000A7F8BDE81040802000F0A2B872B6FEE754
:10111000014600200A0A00D008204FF2F0021142D6
:1011200001D040F004004CF6CC42114201D040F016
:1011300002004AF6AA22114201D040F00100704795
:10114000704700F081B9000070B515460C4608469E
:10115000FFF7DEFF002B0FD0084941F82030204672
:1011600001F088FB04460022294600F01BFA2046C5
:10117000BDE8704000F008BA70BD0000FC210020FE
:10118000D2B200F066B970B5044690F82000002590
:1011900001280CD0012084F8200094F82160002060
:1011A000012E06D084F820000225284670BD0220BA
:1011B00070BD022684F82160A0632068066826F0CE
:1011C000010606602046FFF774FFE06A00282068E9
:1011D000016802D041F00E0106E021F00401016037
:1011E0002068016841F00A0101602068016841F04F
:1011F00001010160D9E7000070B5044600F02EF946
:101200000546601C02D004480078044400F026F92A
:10121000401BA042FAD370BD2C0000202DE9F04104
:101220000024084F0646012505FA04F0304203D099
:1012300057F8240000B18047641CE4B2102CF3D3AB
:10124000BDE8F0813C2200200A20FFF7D5BF000056
:10125000044910B50A68024202D00860FFF7DEFFB9
:1012600010BD0000140401402DE9F84FDFF8B891DB
:101270000024A9F1040B23460F2709F1040AABF15E
:10128000040EC9E00125A5402A40AA427DD1674E3F
:10129000D1F804C0ACEB0608B44532D014DCBCF184
:1012A000030F3AD009DCBCF1000F2AD0BCF1010FCA
:1012B0001CD0BCF1020F31D11DE0BCF1110F17D0D1
:1012C000BCF1120F2AD119E0B8F5881F19D006DC3D
:1012D000B8F5803F15D0B8F5801F1FD111E0B8F5E3
:1012E000001F0ED0B8F5041F18D10AE0CB6815E036
:1012F000CB681B1D12E0CB6808330FE0CB680C33C2
:101300000CE08B682BB1012B4FF0080303D0456133
:1013100004E0042302E0056100E00023FF2A01D875
:10132000064601E000F104064FEA840501D9A5F163
:101330002005D6F8008007FA05FC28EA0C0803FA15
:1013400005F548EA0508C6F800804D68ED0062D54D
:10135000374DAE6946F00106AE61AD6924F0030673
:1013600005F001050095334D06EB050CDCF808503F
:10137000A607360F07FA06F825EA0805DFF8B88051
:10138000404503D14FF0000817E044E0DFF8AC809F
:10139000404502D14FF001080FE0DFF8A48040453E
:1013A00002D14FF0020808E0DFF89880404502D1F2
:1013B0004FF0030801E04FF0040808FA06F848EA85
:1013C0000508CCF808804D68D9F80060ED024D465C
:1013D00001D5164300E096432E604D68DAF80060B0
:1013E000AD02554601D5164300E096432E604D6888
:1013F000DBF80060AD035D4601D5164300E096437F
:101400002E604D68DEF80060ED03754601D5164389
:1014100000E096432E60641C0D682A46E5407FF488
:1014200031AFBDE8F88F0000080401400000111042
:10143000001002400000014000080140000C014083
:1014400000100140001401408068084000D00120D5
:1014500070470AB1016170470904FBE701488068E1
:10146000704700002C00002070B5040004D094F8F0
:101470004100002510B106E0012070BD84F8405005
:10148000204601F049F9242084F841002068C16811
:1014900021F40051C160204602F016FE2068016967
:1014A00021F4904101612068416921F022014161EC
:1014B0002068416941F0080141612068C16841F438
:1014C0000051C1606564202084F8410084F8420026
:1014D0006563002070BD00000248816802781144F5
:1014E000816070472C000020074810B5016841F06A
:1014F00010010160032000F075F80F2000F006F8DD
:1015000000F024F8002010BD0020024070B50D4D01
:1015100004464FF47A712878B1FBF0F00A49096863
:10152000B1FBF0F000F0EAFE48B9102C07D200221F
:101530002146501E00F036F800206C6070BD01207E
:1015400070BD00002C000020380000200C4808B5B9
:10155000816941F001018161816901F0010100911E
:10156000C16941F08051C161C06900F080500090B4
:101570000448416821F0E06141F00071416008BD1C
:101580000010024000000140002809DB00F01F02AB
:10159000012191404009800000F1E020C0F80011D5
:1015A00070470000F0B40E4B1B680C46C3F30223D7
:1015B000C3F10705042D00D90425191D072901D2FF
:1015C000002300E0DB1E012606FA05F1491E21403A
:1015D00099409E40761E16403143F0BC02F00ABE90
:1015E0000CED00E0064900F0070208684FF6FF0323
:1015F000184040EA0220034A104308607047000088
:101600000CED00E00000FA052DE9F0470F4605005B
:1016100061D0434E306800F00700B84209D230680C
:1016200020F0070038433060306800F00700B8420F
:1016300051D128683B4C810712D5400703D560681B
:1016400040F4E06060602878000703D5606840F4EB
:10165000605060606068A96820F0F0000843606036
:101660002878C00728D06868012810D0216802288F
:1016700010D0890700292EDA616821F003010143A7
:101680006160FFF7EBFE804641F288390DE021688A
:101690008903EFE78901EDE7FFF7E0FEA0EB080122
:1016A000494502D90320BDE8F0876068696800F009
:1016B0000C00B0EB810FEFD1306800F00700B842AA
:1016C0000BD9306820F0070038433060306800F0F4
:1016D0000700B84201D00120E5E72878400705D58A
:1016E0006068E96820F4E0600843606028780007DB
:1016F00006D56068296920F4605040EAC100606046
:1017000000F038F86168084AC1F30311515CC84021
:101710000649086006480068FFF7F8FE0020C2E7A7
:1017200000200240001002405A4B00083800002000
:10173000300000200448054900684968044AC1F3A4
:101740000221515CC8407047380000200010024060
:101750006A4B00080448054900684968044AC1F317
:10176000C221515CC8407047380000200010024080
:101770006A4B00080F4A516801F00C00042803D09E
:10178000082803D00C4870470C4870470C48C1F338
:101790008343C903C05C0AD55168094AC1F340417B
:1017A000921E515C054A5043B0FBF1F07047054969
:1017B000484370470010024000127A000024F400F1
:1017C0004A4B000800093D002DE9F84F040070D095
:1017D0002078C04DC00749D06868C0F38100012857
:1017E00007D06868C0F38100022809D16868C00387
:1017F00006D52868800339D560680028E7D035E031
:101800006068B0F5803F0BD010B1B0F5A02F11D0BB
:10181000286820F480302860286820F4802002E0C6
:10182000286840F480302860606890B1FFF716FEA9
:1018300006460AE0286840F480202860F0E700BFF0
:10184000FFF70CFE801B642873D828688003F7D547
:101850000CE0FFF703FE064605E000BFFFF7FEFDC4
:10186000801B6428F0D828688003F7D420789A4E2B
:1018700080074FF001094FF0000839D5686810F073
:101880000C0F07D06868C0F38100022809D168688E
:10189000C00306D42868800714D52069012808D120
:1018A00010E02069B0B1C6F80090FFF7D7FD0746F9
:1018B00005E00AE1FFF7D2FDC01B0228C4D8286862
:1018C0008007F7D52868616920F0F80040EAC10078
:1018D00028600DE0C6F80080FFF7C0FD074604E071
:1018E000FFF7BCFDC01B022823D828688007F7D467
:1018F000207800072CD57948A169D9B1C0F80090AB
:10190000FFF7ACFD074604E0FFF7A8FDC01B022867
:101910000FD8686A8007F7D571484FF4FA5100680C
:10192000B0FBF1F0009000BF0098411E0091FAD288
:101930000EE080E0C0F80080FFF790FD074604E06D
:10194000FFF78CFDC01B022875D8686A8007F7D4A2
:101950002078400760D5E8690027C00008D4E8690E
:1019600040F08050E861E869012700F08050009065
:101970005C480168C90513D40168834641F480714D
:101980000160FFF76BFD824606E000BFFFF766FDD2
:10199000A0EB0A0064284ED8DBF80000C005F5D59E
:1019A000E06801280AD008B1052813D0286A20F081
:1019B00001002862286A20F0040002E0286A40F052
:1019C00001002862E06841F2883B98B1FFF746FDCC
:1019D00082460BE0286A40F004002862EEE700BF70
:1019E000FFF73CFDA0EB0A0159455AD8286A800749
:1019F000F6D50CE0FFF732FD824605E0FFF72EFD3D
:101A0000A0EB0A0159454CD8286A8007F6D41FB1CB
:101A1000E86920F08050E861E06988B36968C1F343
:101A20008101022944D00228C6F8608004D0FFF763
:101A300015FD044638E034E0FFF710FD074604E0EA
:101A4000FFF70CFDC01B02282BD828688001F7D4B3
:101A5000206AB0F5803F05D16868A16820F40030A5
:101A600008436860D4E908010843696821F47411E7
:101A700008436860C6F86090FFF7F0FC044606E093
:101A800025E000BFFFF7EAFC001B022809D8286800
:101A90008001F7D51BE000BFFFF7E0FC001B022828
:101AA00002D90320BDE8F88F28688001F4D40EE045
:101AB0000128F7D06868226A00F48031914204D18D
:101AC000616A00F47010884201D00120EAE700202A
:101AD000E8E7000000100240000042428004424259
:101AE000380000200070004070B5044601F0F4F9A1
:101AF000022811D0204601F0EFF9084D05EB401007
:101B00008069002808D0204601F0E6F905EB401076
:101B10008069BDE87040004770BD00007C22002055
:101B200070B5040009D0606A002540B12561656187
:101B3000A56294F8510040B10CE0012070BD6068CE
:101B4000B0F5827FF4D0E561F2E784F8505020468A
:101B500000F040F8022084F851002068016821F06C
:101B600040010160A088218900F4827001F40441E1
:101B70000843A18901F400610843217C01F00201BE
:101B80000843217D01F001010843218B01F400711C
:101B90000843217F01F03801084394F8201001F038
:101BA00080010843218D01F4005108432168086039
:101BB000A069042101EA1040216848602068C169D9
:101BC00021F40061C1616565012084F851000020A5
:101BD00070BD000030B585B00024009401940294DB
:101BE0000394254D0368254802210322AB421AD1F4
:101BF000836943F480538361836903F480530493BE
:101C0000836943F00403836180691D4D00F0040083
:101C10000490A020CDE90001039269462846FFF711
:101C200023FB40201EE0174DAB4222D1C36943F491
:101C30008043C361C36903F480430493836943F021
:101C4000080383618069104D00F0080004904FF490
:101C50003040CDE90001039269462846FFF704FBB6
:101C60004FF48040CDE90004694628460294FFF70E
:101C7000FBFA05B030BD000000300140001002400A
:101C80000008014000380040000C014070B50446D7
:101C900001F022F9022811D0204601F01DF9084D6B
:101CA00005EB40104068002808D0204601F014F9E8
:101CB00005EB40104068BDE87040004770BD000073
:101CC0007C22002070B5044601F006F9022811D0EC
:101CD000204601F001F9084D05EB4010006900288D
:101CE00008D0204601F0F8F805EB40100069BDE887
:101CF0007040004770BD00007C2200202DE9F84FA5
:101D0000984616468A460446FFF7A8FB814694F893
:101D1000510001281ED1BAF1000F73D0002E71D0EE
:101D200094F85000012815D0012784F85070032042
:101D300084F8510000256565C4F830A0A686E686C3
:101D4000A563A587E58765642564A068B0F5004FA5
:101D500003D00CE00220BDE8F88F2068016821F074
:101D6000400101602068016841F480410160206801
:101D70000168490603D4016841F040010160E06850
:101D8000B0F5006F606803D048B3012E27D047E05C
:101D900008B1012E1FD1206B21680088C86006E0C1
:101DA00020688168890709D5216B0988C160206B8B
:101DB000801C2063E08E401EE0860CE0FFF74EFBA7
:101DC000A0EB0901414503D3B8F1FF3F03D035E053
:101DD000B8F1000F32D0E08E0028E1D123E0206B73
:101DE00021680078087306E02068816889070AD5B1
:101DF000216B09780173206B401C2063E08E401E2C
:101E0000E0860DE02BE0FFF729FBA0EB090141453F
:101E100003D3B8F1FF3F03D010E0B8F1000F0DD0AD
:101E2000E08E0028E0D14A464146204601F039F8CC
:101E300008B120206065A06830B109E084F85170D5
:101E400084F85050032086E72068C16880680090BD
:101E500084F8517004F8505F60680028F3D00120C6
:101E600079E72DE9FF4F81B01D46934604464FF0B8
:101E700001090E9EFFF7F2FA074694F851006168D7
:101E8000012806D0B1F5827F3CD1A168C9BB0428E6
:101E900038D10298002871D0BBF1000FFBD0002D83
:101EA000F9D094F8500001282CD04FF0010A84F8A2
:101EB00050A094F85100042802D0052084F8510065
:101EC0004FF00008C4F85480C4F838B0E587A587FF
:101ED00002992163E586A586C4F84080C4F8448051
:101EE00020680168490603D4016841F0400101609F
:101EF000E068B0F5006F606808D0F0B3012D49D0FC
:101F000081E0FFE7022005B0BDE8F08F08B1012DA8
:101F100039D1206B21680088C860206B801C206349
:101F2000E08E401EE0862EE02068816889070FD58C
:101F3000E18E69B1B9F1010F0AD1216B0988C16045
:101F4000206B801C2063E08E401EE0864FF000096D
:101F500020688168C9070CD0E18F51B1C068A16BBE
:101F60000880A06B801CA063E08F401EE0874FF0CC
:101F70000109FFF773FAC01B01E00BE067E0B04214
:101F800001D3701C50D1E08E0028CDD1E08F002805
:101F9000CAD13EE0206B216800780873206B401C9A
:101FA0002063E08E401EE0862DE02068816889076E
:101FB0000FD5E18E69B1B9F1010F0AD1216B097812
:101FC0000173206B401C2063E08E401EE0864FF0C2
:101FD000000920688168C9070CD0E18F51B1C06841
:101FE000A16B0870A06B401CA063E08F401EE087CF
:101FF0004FF00109FFF732FAC01BB04202D3701C48
:1020000001D011E086B1E08E0028CED1E08F00280B
:10201000CBD13A463146204600F043FF50B1202054
:10202000606584F8508012E084F851A084F85080F4
:10203000032068E7A06818B92068C168806800902C
:1020400084F851A084F85080606D0028F1D0012000
:1020500059E7000070B5044690F851006568012802
:1020600006D0B5F5827F3AD1A568A5BB042836D144
:1020700091B38AB383B394F8500001282FD0012084
:1020800084F8500094F85100042802D0052084F808
:102090005100002565652163A386E386A263A387BB
:1020A000E3872564656494F85100042819D0E16C35
:1020B0002748C8622748E16C8862E16C26480863BB
:1020C000E06C4563E38F2168A26B0C31E06CFFF795
:1020D0005AF800BB0AE002E0FFE7012070BD0220D1
:1020E00070BDE16C1D48C8621D48E4E72068416886
:1020F00041F001014160A06CC562A06C8562A06CDA
:102100000563A06C4563E38E2268216B0C32A06CE2
:10211000FFF739F830B1606D40F01000606584F869
:102120005050DAE720680168490603D4016841F09D
:102130004001016084F850502068416841F020015E
:1021400041602068416841F002014160002070BD9B
:10215000152D0008ED2D0008DF2C0008012D0008CA
:102160001F2D000870B5044690F8510001281CD1BD
:10217000C9B1C2B194F85000012816D0012084F8EA
:102180005000032084F85100002565652163A28674
:10219000E286A56365642564A587E587A068B0F538
:1021A000004F04D00DE0012070BD022070BD2068FA
:1021B000016821F0400101602068016841F480411C
:1021C0000160A16C1748C862A16C17488862A16CB5
:1021D00016480863A06C4563E38E2268216B0C32BD
:1021E000A06CFEF7D0FF30B1606D40F0100060656C
:1021F00084F85050D7E720680168490603D4016885
:1022000041F04001016084F850502068416841F07D
:10221000200141602068416841F0020141600020D6
:1022200070BD00000B2D0008892D0008DF2C000870
:1022300010B500F051FE022808D0054901EB40100E
:102240000068002802D0BDE81040004710BD000023
:102250007C22002070B5044600F03EFE022811D01A
:10226000204600F039FE084D05EB4010C0680028FC
:1022700008D0204600F030FE05EB4010C068BDE8F5
:102280007040004770BD00007C22002070B50446FD
:1022900000F022FE022811D0204600F01DFE084D5D
:1022A00005EB40108068002808D0204600F014FE9E
:1022B00005EB40108068BDE87040004770BD00002D
:1022C0007C22002070B5044600F006FE022811D0E2
:1022D000204600F001FE084D05EB40104069002843
:1022E00008D0204600F0F8FD05EB40104069BDE83D
:1022F0007040004770BD00007C22002010B5401ED9
:10230000B0F1807F01D3012010BD4FF0E024606167
:102310000F21601701F06EFF0020A06107202061EF
:10232000002010BD10B590F83C20012A22D00122D7
:1023300080F83C20CA688C6822F4407222434C68C2
:1023400022F4806222430C6822F4006222430C696A
:1023500022F4805222434C6922F400522243C9697C
:10236000002322F480420A4301684A6480F83C302A
:10237000002010BD022010BD70B590F83C20012A4D
:1023800026D0012480F83C40022280F83D200368DA
:102390005A689D6822F070060A6832435A600D4BF5
:1023A00002689A4208D0B2F1804F05D00A4B9A4297
:1023B00002D00A4B9A4204D1496825F080031943A0
:1023C000916080F83D40002180F83C10084670BDC7
:1023D000022070BD002C01400004004000080040B5
:1023E00010B5040003D094F83D0010B107E00120BF
:1023F00010BD002084F83C00204600F01FF80220A9
:1024000084F83D00211D206801F024FD012084F89E
:10241000460084F83E0084F83F0084F8400084F8C9
:10242000410084F8420084F8430084F8440084F8B2
:10243000450084F83D00002010BD000008B500688C
:102440000649884208D10648816941F400618161EA
:10245000806900F40060009008BD0000002C01407D
:102460000010024070B5044690F83C000025012899
:1024700017D0012684F83C60022084F83D002068D3
:10248000826822F0770222F47F4282600868502836
:1024900038D00DDC20284FD005DC90B3102811D1A6
:1024A0004AE0022070BD302846D040280AD13BE0E7
:1024B00060282FD070280DD0B0F5805F03D0B0F524
:1024C000005F12D0012584F83D60002084F83C00B4
:1024D000284670BDCB68D1E90121206801F0F6FCE7
:1024E0002068816841F0770109E0CB68D1E90121DA
:1024F000206801F0EBFC2068816841F48041816034
:10250000E1E719E0CA684968206801F093FD5021AD
:10251000206806E0CA684968206801F09CFD6021D7
:10252000206801F0DDFCCEE7CA684968206801F048
:1025300081FD40212068F4E7226801461046F0E75B
:1025400000B585B0002100910191029103910068CE
:102550000B49884212D10B48816941F00401816125
:102560008069694600F0040004904FF40060009018
:102570000220019003900448FEF776FE05B000BDEE
:10258000002C0140001002400008014070B50446D4
:1025900090F83C0000260D4601280FD0012084F859
:1025A0003C006AB1042A1DD0082A2FD00C2A3FD043
:1025B0000126002084F83C00304670BD022070BD2A
:1025C000206801F095FC2068816941F00801816173
:1025D0002068816921F004018161206881692A698C
:1025E000114311E0206801F0ABFC2068816941F4DF
:1025F000006181612068816921F4806181612068C6
:1026000081692A6941EA02218161D2E7206801F0EB
:10261000C3FC2068C16941F00801C1612068C1693B
:1026200021F00401C1612068C1692A69114311E0E8
:10263000206801F0DDFC2068C16941F40061C161DE
:102640002068C16921F48061C1612068C1692A697B
:1026500041EA0221C161ACE710B5040003D094F84F
:102660003D0010B107E0012010BD002084F83C00BF
:10267000204600F01EF8022084F83D00211D20684D
:1026800001F0E8FB012084F8460084F83E0084F85D
:102690003F0084F8400084F8410084F8420084F848
:1026A000430084F8440084F8450084F83D0000208D
:1026B00010BD704770B5040004D094F841000025A7
:1026C00010B106E0012070BD84F84050204600F0B3
:1026D00023F8242084F841002068C16821F40051C7
:1026E000C160204601F0F0FC2068016921F49041AE
:1026F00001612068416921F02A0141612068C168B7
:1027000041F40051C1606564202084F8410084F8E0
:1027100042006563002070BD30B585B00024009490
:10272000019402940394224D036822490322224813
:10273000AB4216D18B6943F480438B618B6903F400
:10274000804304938B6943F004038B61896903928E
:1027500001F0040104914115009112210191694693
:1027600021E0164DAB4220D1CB6943F40033CB615D
:10277000CB6903F4003304938B6943F004038B614A
:102780008969039201F0040104910421009102215E
:10279000019169460546FEF767FD0820CDE9000472
:1027A000694628460294FEF75FFD05B030BD000083
:1027B0000038014000100240000801400044004081
:1027C0002DE9F843044690F84100984616460D4618
:1027D000202802D00220BDE8F88385B17EB1002018
:1027E0006064212084F84100FEF738FEA68481460B
:1027F000E684A0682027B0F5805F02D003E00120C6
:10280000E9E7206910B12E4600250EE000260CE015
:102810008021204601F0B4FCA8B9C6B116F8010B1E
:1028200021684860E08C401EE084E08C4B464FF00D
:102830000002CDF800800028EAD14FF04001204688
:1028400001F09EFC40B184F841700320C3E735F8E5
:10285000020BC0F30800E3E784F841700020BAE7F8
:10286000FEE710B5FEF740FEFEF76AFCBDE810403B
:1028700001F0AABA00B5FEF74BFC012801D80620EA
:1028800000BD032801D8072000BD052801D8082075
:1028900000BD072801D8092000BD092801D80A2059
:1028A00000BD0F2801D8172000BD282000BD000062
:1028B0002DE9F04186B00026384800960196029630
:1028C0000396816941F020018161816901F0200155
:1028D0000491816941F004018161816901F0040181
:1028E0000491816941F00801816180692C4F00F0F9
:1028F00008000490002210213846FEF7AAFDDFF8F8
:10290000A480002219214046FEF7A3FD01241020D7
:10291000CDE90004022569463846CDE90245FEF7B7
:10292000A3FC0094694640460194CDE90245FEF7B8
:102930009BFC200300901C48CDE9010669463846FF
:10294000FEF792FC18208DE8310069464046039559
:10295000FEF78AFCE02000901448CDE901056946A5
:102960004046FEF781FC2002CDE90006694602954B
:102970004046FEF779FC002205211720FEF712FEE3
:102980001720FEF701FE002211462820FEF70AFE5E
:102990002820FEF7F9FD06B0BDE8F08100100240E6
:1029A00000080140000C014000002110000011103F
:1029B000104810B50E4901604FF48271416000214A
:1029C0008160C1604FF400720161C0E905121822F4
:1029D000C0E90721416281620A21C162FFF7A0F8C4
:1029E000002803D0BDE81040FEF790BB10BD0000EA
:1029F00000300140740000200F4810B50D490160FF
:102A00004FF48271416000218160C1604FF4007217
:102A10000161C0E90512C1610162416281620A215E
:102A2000C162FFF77DF8002803D0BDE81040FEF733
:102A30006DBB10BD00380040CC00002010B596B032
:102A400000240F9410941194129413941C2108A83C
:102A50001494FDF7D9FD20216846FDF7D5FD2748E0
:102A60002549C0E900144FF6FF71C0E90241046135
:102A700044618461FFF7B4FC08B1FEF747FB4FF4F3
:102A800080500F900FA91D48FFF7ECFC08B1FEF72E
:102A90003DFB1A48FFF7E0FD08B1FEF737FB139442
:102AA00013A916481494FFF767FC08B1FEF72EFB34
:102AB0006020CDE908040A940C940D940C2208A916
:102AC0000E480E94FFF762FD08B1FEF71FFB00945D
:102AD0004FF40050CDE904400294019403946946F8
:102AE00006480794FFF71EFC08B1FEF70FFB0348EA
:102AF000FFF726FD16B010BD002C01402401002078
:102B00000C4810B50A4901604FF4E13141600021E1
:102B100081600822C160C0E904128161C161FEF7D1
:102B2000A3FC002803D0BDE81040FEF7EFBA10BDAB
:102B3000003801406C0100200C4810B50A490160C2
:102B40004FF4E1314160002181600C22C160C0E995
:102B500004128161C161FFF7ADFD002803D0BDE81B
:102B60001040FEF7D3BA10BD00440040B40100206D
:102B7000FEE7FEE770B50C4C0120002560700B48A5
:102B8000257005222146036E881D98472178A01DD7
:102B90000844457006A0FDF729FBA11DBDE8704063
:102BA00006A0FDF723BB000000000020784B0008C2
:102BB0004F6E5278446F6E650D0A00002564000068
:102BC000064910B50320487005A0FDF70FFB084823
:102BD00008490069C96DBDE81040084700000020A1
:102BE0005258453C3E3E3E3E3E3E3E3E0A0D0000B3
:102BF000344B0008784B0008064910B50220487095
:102C000005A0FDF7F3FA0A480A49C068C96DBDE896
:102C100010400847000000203C3E3E3E3E3E3E3E07
:102C20003E4F6E527854696D656F75740A0D0000E1
:102C3000344B0008784B000870B50A4D04206870CA
:102C400009A0FDF7D3FA0D4CA9880023666D1A463A
:102C50000846B0470A48636E05214268BDE87040E7
:102C600008A01847000000203C3E3E3E3E3E3E3E4F
:102C70003E4F6E5478446F6E650A0D00784B000825
:102C8000344B0008313233343500000070B50A4D42
:102C90000520687009A0FDF7A9FA0C4CA98800234B
:102CA000666D1A460846B0470948636E052182687A
:102CB000BDE8704007A01847000000203C3E3E3EA3
:102CC0003E3E3E3E3E5458450A0D0000784B0008FB
:102CD000344B00083132333435000000704710B5F2
:102CE000406A01684A6822F003024A60416D41F07F
:102CF00010014165012180F85110FEF7F5FE10BD6D
:102D000010B5406AFEF7DEFF10BD10B5406AFFF750
:102D1000A1FA10BD10B5406AFFF7D4FA10BD70B526
:102D20000546446AFEF79AFB02462868006880065A
:102D300026D42068416821F020014160A06818B9BC
:102D40006068B0F5827F16D02068416821F00101EB
:102D500041606421204600F076F808B120206065CB
:102D60000020E087012084F85100606D40B12046CA
:102D7000FEF7BAFE70BD2068416821F00301E7E765
:102D80002046FEF783FF70BD38B50546446AFEF75E
:102D900065FB024628680068800623D420684168E5
:102DA00021F0200141602068416821F0020141606A
:102DB0006421204600F075F818B1606D40F02000E5
:102DC0006065A068002118B92068C268806800901A
:102DD000E186012084F85100606D18B12046FEF7AD
:102DE00083FE38BD2046FFF723FA38BD70B505468F
:102DF000446AFEF733FB02462868006880061ED44A
:102E00002068416821F0200141606421204600F0E3
:102E100048F818B1606D40F0200060652068416896
:102E200021F0030141600020E086E087012084F862
:102E30005100606D18B12046FEF756FE70BD204669
:102E4000FFF724FA70BDF8B5044640684FF482736A
:102E5000984217D1A0684FF48065B0F5004F01D0BB
:102E6000A8420FD12068066826F040060660606818
:102E7000984207D1A068A84204D100920B460022D4
:102E8000012103E000920B4600228021204600F041
:102E90002DF8002804D0606D40F02000606503200C
:102EA000F8BDF8B515460E460B46009204460122C1
:102EB000022100F01BF840B9334600228021204651
:102EC000009500F013F8002804D0606D40F0200059
:102ED00060650320F8BD000000680349884201D105
:102EE0000020704702207047003001402DE9F84370
:102EF0001E46914688460446089DFEF7AFFA401BE1
:102F0000351AFEF7ABFA074625480068C0F3CB3008
:102F1000684338E0701C37D0FEF7A0FAC01BA84207
:102F200003D215B1009860B32CE02068416821F00D
:102F3000E00141606068B0F5827F0BD1A068B0F518
:102F4000004F02D0B0F5806F04D12068016821F0F5
:102F500040010160A06AB0F5005F09D120680168F6
:102F600021F4005101602068016841F400510160C2
:102F7000012084F85100002084F850000320BDE8AF
:102F8000F8830025401E00902068816838EA01001F
:102F900004D000214945BDD10020F0E70121F9E727
:102FA000380000207047C0F340114901C0F30012FF
:102FB00041EA0211C0F3C00241EAC201C0F380023B
:102FC00041EA8201C0F3400241EA420108B500F043
:102FD000010001438DF8001001226946892000F0AC
:102FE00017FB08BD08B5010A8DF800108DF8010027
:102FF00002226946972000F00BFB08BD10B54FF484
:10300000AA7000F079FA044640F2531000F074FA06
:1030100044EA002010BD000070B5204A002001469F
:103020005278032A39DA002A37D0012A35D140F6FE
:10303000541000F061FA044640F6551000F05CFAB6
:10304000054640F6561000F057FA210441EA0521E2
:103050000143C1F3130400F035F801F042FC0246CD
:103060000B4600200E4901F0B7FA00220D4B01F08B
:1030700063FC05460E462046B4F5002F01D3A4F5A7
:10308000801001F02EFC084A084B01F055FC2A463E
:103090003346BDE8704001F09FBA70BD3C0000208F
:1030A0000000994000408F40CDCCCCCCCCCCF83F38
:1030B00008B502226946152000F0E8F9BDF80000C5
:1030C00040BA08BD0949002089780A290BD018297F
:1030D00007D0262903D0342900D105487047054878
:1030E0007047054870470548704700003C000020C5
:1030F00075190300EA320600D4650C00A8CB18004D
:1031000001480078704700003C0000201CB50446D0
:10311000052269461D2000F0B9F9804840782070EA
:10312000032865D00FDCC0B1012815D19DF800003F
:10313000404200EBD070401060709DF80100802884
:1031400019D280081DE004287DD00F2804D100206A
:103150002060A0800F2020701CBD9DF80000404220
:1031600000EBD070401060709DF80100404200EB11
:10317000D070401005E0A0F58070C11700EB917091
:103180008010A0709DF802008109E07861F30000D2
:10319000E0709DF80210490961F34100E0709DF86C
:1031A0000210090961F38200E0709DF80210C9085D
:1031B00061F3C300E0709DF80210890861F3041008
:1031C000E0709DF80210490861F34510E0709DF829
:1031D000021061F38610E0709DF803004109207928
:1031E00061F3000020719DF8031061F341008DE050
:1031F0009DF80000404200EBD070401060709DF8D8
:103200000100404200EBD0704010A0709DF8020019
:103210008109E07861F30000E0709DF8021049092F
:1032200061F34100E0709DF80210090961F382002A
:10323000E0709DF80210C90861F3C300E0709DF8CA
:103240000210890800E025E061F30410E0709DF8A9
:103250000210490861F34510E0709DF8021061F317
:103260008610E0709DF803008109207961F3010068
:1032700020719DF80310490961F3820020719DF8C7
:103280000310090961F3C30020719DF8031061F375
:1032900004103BE09DF80000404200EBD07040106D
:1032A00060709DF80100404200EBD0704010A070AB
:1032B0009DF802008109E07861F30000E0709DF85C
:1032C0000210490961F34100E0709DF802100909FC
:1032D00061F38200E0709DF80210C90861F3C30039
:1032E000E0709DF80210890861F30410E0709DF809
:1032F0000210490861F34510E0709DF8021061F377
:103300008610E0709DF8030000F0010020719DF828
:10331000040000F0070060711CBD00003C000020AC
:1033200001484078704700003C000020F8B50C468A
:10333000064615466946204600F01EF82278AA4245
:1033400001D90120F8BD31469DF8000000F068F871
:103350000020F8BD08B500208DF800000122694664
:103360001F2000F093F89DF80000404200EBD07061
:1033700040F3470008BD0000F8B50D4604460222A0
:103380006946172000F082F80C4E707801280AD1A7
:1033900040F6031000F0B0F8C00904D040F6011068
:1033A00000F0AAF805E0707804289DF8000000D12C
:1033B000801C20709DF801002870F8BD3C000020A2
:1033C00008B500208DF8000001226946C02000F0F9
:1033D0005DF89DF8000008BD70B5074D4FF4807191
:1033E0002846FDF7AEFE044680212846FDF7A9FEDB
:1033F00044EA4000C0B270BD000C014010B5044664
:1034000000F0BAF82046BDE8104000F001B8000016
:103410000022036880210148FDF796BE000C0140A0
:103420002DE9F0410E46014615481446D51C1B22D5
:1034300002704170002181700B4603E0C2185B1CD2
:10344000D1709BB2A342F9D300F0B0F80D4F002227
:1034500010213846FDF794FE2A460B49084800F033
:10346000A3FC09492246C91C3046FDF766F8012233
:1034700010213846FDF784FEBDE8F04100F096B813
:10348000FC01002000080140FB1100202DE9F04163
:103490000E460146901C85B2144814460170002166
:1034A00041700B4603E0C2185B1C91709BB2A342B3
:1034B000F9D300F07BF80E4F002210213846FDF7BB
:1034C0005FFE2A460B49094800F06EFC0949224676
:1034D000891C3046FDF731F8012210213846FDF7EE
:1034E0004FFEBDE8F04100F061B80000FC01002093
:1034F00000080140FB11002008B50122694600F0D8
:1035000003F89DF8000008BD2DE9F0410E46111D9D
:10351000164B8DB219211970010A5970987000214B
:103520001446D970084603E01A18401C117180B285
:10353000A042F9D300F03AF80D4F0022102138468E
:10354000FDF71EFE2A460B49084800F02DFC0949EC
:103550002246091D3046FCF7F0FF012210213846B3
:10356000FDF70EFEBDE8F04100F020B8FC010020A0
:1035700000080140FB11002010B51420FDF73CFEAF
:10358000094C002201212046FDF7FAFD3220FDF70B
:1035900033FE012211462046FDF7F2FDBDE8104042
:1035A0001420FDF729BE0000000C014070B5054D48
:1035B0004FF4807421462846FDF746FF0128F9D0D4
:1035C00070BD0000000C014070B50F481A23941C18
:1035D00000F8013B002300F8013BFCF7AEFFFFF7CA
:1035E000E5FF0A4D002210212846FDF7C9FD2146BE
:1035F000054800F0CDFB012210212846FDF7C0FD53
:10360000BDE87040FFF7D2BFFC0100200008014078
:103610002DE9F0410546501C1446884686B2FFF756
:10362000C5FF0F4F002210213846FDF7A9FD0D48B8
:103630002246414600F8015BFCF77FFF314609480E
:1036400000F0A6FB012210213846FDF799FD842DDC
:1036500003D0BDE8F041FFF7A9BFBDE8F08100004D
:1036600000080140FC01002013B5012201A900F06F
:1036700001F81CBD70B50346D01C84B20F48182554
:1036800000F8015B1D0A00F8015B00F8013BFCF744
:1036900054FFFFF78BFF0A4D002210212846FDF74B
:1036A0006FFD2146054800F073FB012210212846DA
:1036B000FDF766FDBDE87040FFF778BFFC01002014
:1036C000000801400249C86001F10800FFF796BEFA
:1036D0003C0000200348C17811B1012101717047FD
:1036E00000F002B83C00002070B5514C2078002852
:1036F00072D0E07830B1207900286DD072B6002009
:10370000207162B66678FFF7D3FC05464FF6FF706E
:10371000FFF768FC2EB1012E40D0032E01D0042EFD
:103720005AD1207804286FD0052855D1A80714D580
:10373000680605D5E06880B1816971B1022006E0B4
:103740002807E06805D540B1816931B1012088477B
:1037500003E010B1406800B18047680704D5E06815
:1037600010B1806800B18047280705D5E06818B11E
:10377000816909B1012044E0680458D5E068002857
:1037800055D0406905E0680451D5E06800284ED066
:10379000006900284BD0BDE870400047207804281D
:1037A00032D005280DD0062841D1E804E4D5A8047C
:1037B000E06833D500283AD0C169002937D001200C
:1037C00032E0A8070DD56806E06806D548B18169E2
:1037D00039B10220884704E029E010B1406800B107
:1037E0008047E80604D5E06810B1C06800B18047A2
:1037F000A806C1D5E0680028BED081690029BBD0E9
:1038000000208847B8E7FFE7E807BCD0E068002859
:10381000B9D000680028B6D08047B4E7002806D0A9
:10382000C169002903D00020BDE87040084770BD81
:103830003C00002010B5144600F080F92046BDE899
:10384000104000F067BA01B5012269469E20FFF7DB
:10385000DFFE08BD08B52138010A8DF800108DF88B
:103860000100022269469820FFF7D2FE08BD10B57C
:103870000446010E40F6CF10FFF7F6FEC4F30741F1
:103880004FF41D60FFF7F0FEC4F3072140F6D1109E
:10389000FFF7EAFEE1B2BDE8104040F6D210FFF7B4
:1038A000E3BE00000148FFF7E2BF0000D6BE898EEC
:1038B00008B502228DF800008DF8011069468F20AE
:1038C000FFF7A6FE08BD000010B500221146C52076
:1038D000FFF79EFE01490620087010BD3C00002045
:1038E00001B5012269468820FFF792FE01490620B2
:1038F000087008BD3C00002008B5010A8DF80010D2
:103900008DF801000548407808B1032805D102224E
:10391000694640F6C610FFF7ADFE08BD3C0000202A
:1039200008B5010A8DF800108DF8010005484078AF
:1039300008B1032805D10222694640F6C810FFF7F6
:1039400099FE08BD3C0000201CB5040A8DF800401B
:103950008DF80100080A8DF80200100A8DF80400A5
:103960008DF80520180A8DF806008DF803108DF8E3
:103970000730082269468D20FFF74AFE1CBD000073
:1039800010B500221146C120FFF742FE0149032075
:10399000087010BD3C00002001490020C87070472D
:1039A0003C00002001B5012269469B20FFF730FE54
:1039B00008BD000038B5234D044600786978884278
:1039C00001D000F0ADF8207803281DD003DC38B119
:1039D000012822D10CE0042825D00F281DD12AE08F
:1039E00060788DF80000A0788DF80100E07812E092
:1039F00020798DF8000060798DF80100A0798DF8AC
:103A000002006079A87008E0E0798DF80000207A63
:103A10008DF80100607A8DF80200032269468B2040
:103A2000FFF7F6FD38BDA07A8DF80000E07A8DF83A
:103A30000100207BEFE700208DF800008DF80100E9
:103A4000E9E700003C0000201CB53449044600783A
:103A50004978884201D000F063F8217800200329DA
:103A600035D003DC39B101292BD118E0042942D02B
:103A70000F2926D14CE060788DF80000A0788DF8F1
:103A80000100E0788DF8020020798DF8030060795C
:103A90008DF80400A0798DF80500E0790FE0217A17
:103AA0008DF80010617A8DF80110A17A8DF802105E
:103AB000E17A8DF80310217B8DF804102BE08DF84E
:103AC0000600072269468C20FFF7A2FD1CBD607B23
:103AD0008DF80000A07B8DF80100E07B8DF80200DE
:103AE000207C8DF80300607C8DF80400A07C8DF8AC
:103AF0000500E07CE3E7217D8DF80010617D8DF805
:103B00000110A17D8DF80210E17D8DF8031000E019
:103B100000908DF804008DF80500D0E73C000020EF
:103B200001B505499DF800000122487069468A20C8
:103B3000FFF76EFD08BD00003C0000200A4601466C
:103B40000020FFF741BD000001490120C870704707
:103B50003C00002070B5074D002400BF05EB840039
:103B6000817835F82400FFF77FFD641C24B2002C17
:103B7000F4D070BD724B000801B501226946962051
:103B8000FFF746FD08BD000008B500F0C1FE0022A9
:103B9000094B00F021FD00F077FE010C8DF80010BC
:103BA000010A8DF801108DF8020003226946862073
:103BB000FFF72EFD08BD0000A8CB684008B58DF8C2
:103BC0000000000C010A8DF801108DF802004FF67C
:103BD000FF70FFF707FA032269468220FFF718FDFE
:103BE00001490520087008BD3C0000201CB58DF877
:103BF0000000080A8DF801008DF80210100A8DF8F7
:103C000003008DF80420052269469420FFF700FD8B
:103C10000149052008701CBD3C000020002211460F
:103C2000D520FFF7F5BC0000C107090FC0F3400223
:103C300041EA8201C0F3800208B541EA4201C0F3C3
:103C4000C00001438DF800100449002001220870D3
:103C500069468420FFF7DCFC08BD00003C00002022
:103C600001B5012269468020FFF7D2FC9DF80010C3
:103C7000034811B10221017008BD0121FBE70000DA
:103C80003C0000200346194810B5427832B140F696
:103C9000CF10032A13D0042A22D11EE00522012BC3
:103CA00004D0022B05D0032B1AD105E040F6CE102C
:103CB00018E040F6D31015E040F6D81012E00422C8
:103CC000012B0FD0022B02D0032B09D102E040F6CA
:103CD000D41007E040F6D91004E00422012B01D0F3
:103CE000012010BDFFF7C6FC002010BD3C000020E5
:103CF00070B5044640F6CD152846FFF7FDFB00F0F1
:103D0000F00104F00F0001432846BDE87040FFF7C2
:103D1000ABBC000008B58DF80000000C010A8DF85E
:103D200001108DF802004FF6FF70FFF75BF90322D8
:103D300069468320FFF76CFC01490420087008BD28
:103D40003C00002000221146D220FFF761BC002277
:103D50001146D120FFF75CBC08B512308DF8000089
:103D60008DF80110022269468E20FFF751FC08BD34
:103D70000649497819B1032901D0042904D1014623
:103D800040F6C510FFF770BC704700003C000020F3
:103D9000044A0123537013780A4601460020FDF7B8
:103DA0005DB900004C00002038B5064B01245C7062
:103DB0001B78009313460A4601460020FDF762F97E
:103DC00038BD00004C00002010B5064A022100203A
:103DD000FDF736F90021BDE81040034A0846FDF71B
:103DE0002FB90000CD450008C1450008FDF774BBA0
:103DF00010B590B028216846FCF706FC14210AA8EB
:103E0000FCF702FC01210804CDE9001042000292F7
:103E100002240491CDE907404FF4E0100990684670
:103E2000FDF7D2FC08B172B6FEE70F20CDE90A0417
:103E300000204FF48061CDE90C010E9002210AA808
:103E4000FDF7E2FB002801D072B6FEE710B010BD0E
:103E500070470000F0B50268194B1A4C1A4D4FF02C
:103E60008047984205D0B84203D0A04201D0A84272
:103E700003D122F070064A683243984205D0B84216
:103E800003D0A04201D0A84203D122F44074CA68F2
:103E900022434C6922F08002224302608A68C26297
:103EA0000A688262984201D1096901630121416176
:103EB0000169C90703D0016921F001010161F0BD69
:103EC000002C0140000400400008004010B5846848
:103ED00042EA032224F47F440A432243826010BD55
:103EE000826822F070020A4342F007018160704745
:103EF00030B5036A026A22F00102026242688469F4
:103F000024F073050C682C4323F002058B682B43C7
:103F10000A4DA8420BD123F00805CB6822F4407269
:103F20002B434D6923F0040315438A692A434260F9
:103F3000846149684163036230BD0000002C014088
:103F400030B5026A036A23F0100303624368846990
:103F50000D6824F4E64444EA05248D6822F020022A
:103F600042EA05120B4DA8420ED1CD6822F0800224
:103F700042EA05124D6923F4406343EA85038D69E3
:103F800022F0400243EA850343608461496881630B
:103F9000026230BD002C014030B5036A026A22F48F
:103FA000807202624268C46923F4007324F07305CE
:103FB0000C682C438D6843EA05230C4DA8420ED1B2
:103FC000CD6823F4006343EA05234D6922F440528F
:103FD00042EA05128D6923F4806342EA05124260C9
:103FE000C4614968C163036230BD0000002C014018
:103FF00030B5046A026A22F4805202624268C369E0
:104000000D6823F4E64343EA05238D6824F4005445
:1040100044EA0534064DA84204D14D6922F4804299
:1040200042EA85124260C36149680164046230BD9E
:10403000002C014010B5036A046A24F001040462F4
:10404000846924F0F00444EA021423F00A020A43CB
:104050008461026210BD10B5036A046A24F0100482
:104060000462846923F0A00324F4704444EA023219
:1040700043EA01118261016210BD01680C3151E80F
:10408000002F22F4907241E80023002BF5D1016843
:10409000143151E8002F22F0010241E80023002BE7
:1040A000F5D1016B012909D101680C3151E8002FCC
:1040B00022F0100241E80023002BF5D1202180F8E6
:1040C000421000210163704770B504460068016921
:1040D000E26821F44051114301612169A06808435D
:1040E000616908432168CA6841F20C639A4302433C
:1040F000CA6020684169A26921F44071114341619D
:104100001E492068884202D1FDF724FB01E0FDF73B
:1041100011FB00EBC00101EB00126068642180001C
:10412000B2FBF0F3B3FBF1F36FF018067343B2FB8D
:10413000F0F5B2FBF0F605EB8305322303EB051532
:10414000B5FBF1F5B6FBF1F605F0F00505EB06154C
:10415000B2FBF0F6B2FBF0F0B0FBF1F06FF018023A
:10416000504306EB800003EB0010B0FBF1F0216838
:1041700000F00F002844886070BD00000038014046
:104180002DE9F843984617460D460446089E24E05C
:10419000701C22D0FDF762F9A0EB0800B0421AD8DB
:1041A000CEB12068C168490717D5802D15D0402DA4
:1041B00013D00168C94309070FD40168002540687E
:1041C00000902046FFF759FF0820606484F84050B3
:1041D0000120BDE8F8830320FBE72068006835EA8A
:1041E000000004D00020B842D2D00020F1E7012026
:1041F000F9E7FEE70907090E002804DB00F1E020DB
:1042000080F80014704700F00F0000F1E02080F803
:10421000141D704730380A2801D201207047002051
:104220007047000013B54FF0FF3301226946024882
:10423000FEF7C6FA00981CBDB40100208CB0FDF753
:1042400053F9FFF7D5FDFEF733FBFEF7B1FBFEF7A1
:10425000D3FBFEF7F3FBFEF753FCFEF76DFCFDF717
:1042600079FA0546FDF766FA0446FDF783FA01463A
:104270002B4622467FA0FBF7B9FFFEF7F2FA4FF478
:10428000FA70FCF7B9FF844C844821688847834F53
:104290000C3FB81D3978FCF795F9FFF76DF9804EA2
:1042A0004FF4807529463046FDF7CEF80028F9D145
:1042B0007CA000250068DFF8F081CDE908052A46DA
:1042C000102146464046FDF7C4F84FF06409032329
:1042D00009AA08A97548CDF80090FDF7C2FD012292
:1042E00010213046FDF7B5F89DF822309DF82120C9
:1042F0009DF820106EA0FBF779FF9DF826309DF801
:1043000025209DF824106FA0FBF770FF01268DF883
:104310002860E36932460AA9002098479DF82810D2
:104320006DA0FBF763FF75A17BA0FBF75FFF206B20
:104330008047014685A0FBF759FF8EA0FBF756FF8B
:10434000C0208DF808000A208DF8090007208DF89C
:104350000A0091488DF804600C21067001724572C4
:10436000052181722021C17240210173A16B0020BF
:104370008847E16B9DF804008847216C01A88847B5
:10438000616C85488847A16C844888470021E26CAD
:10439000084690470021226D0D209047A16B002018
:1043A00088479DF8080010F00F0F11D10111491F27
:1043B00040F6251008290BD2DFE801F004040707B6
:1043C000595959591E21A26901E0A2693721904724
:1043D000FFF7E2FA7D7079880023666D1A46084679
:1043E000B0476F48E16D006888470122E36907A97B
:1043F000104698479DF81C106AA0FBF7F7FE46464A
:104400004FEA0907FFF770F96420FCF7F5FED4F8CE
:10441000A8008047010002D065A0FBF7E7FE21A0BD
:1044200000220068CDE9050510213046FDF711F89E
:10443000032306AA05A91D480097FDF712FD0122D6
:1044400010213046FDF705F89DF816309DF815202F
:104450009DF8141016A0FBF7C9FE9DF81A309DF8C0
:1044600019209DF8181017A0FBF7C0FECAE73221EB
:10447000A269ACE7434C4B3A205359533D256C6439
:1044800020415042313D256C6420415042323D254F
:104490006C640D0A00000000784B00080C0000203E
:1044A000000C01404800000000080140740000209A
:1044B00074783A2025303258202530325820253063
:1044C00032580A0072783A2025303258202530328E
:1044D0005820253032580A0052656730303D256437
:1044E0002020286578706563742030783430206F20
:1044F000722030784646290D0A0000004669726D28
:10450000776172652056657273696F6E3A20313734
:1045100030393139410000000A0A0D2020202020C6
:104520005358313238312050696E6720506F6E67B2
:104530002044656D6F204170706C69636174696FB0
:104540006E2E2025730A0A0D000000000A0A0D20B5
:1045500020202020526164696F206669726D776146
:1045600072652076657273696F6E20307825780ADF
:104570000A0D00000A50696E6720506F6E67207246
:10458000756E6E696E6720696E204C4F5241206DCA
:104590006F64650A0D0000005C00002080D29990D5
:1045A000344B00085374617475733D25640A000030
:1045B0004952513D3078253034580D0A0000000032
:1045C00001490020487070474C000020014900203C
:1045D000487070474C0000202DE9C04130B4DFF82E
:1045E000A0C23CEA111418BF3CEA131400F0EC809E
:1045F00081EA03051CEA111444EAD57418BF1CEAC9
:10460000131500F0C780A4EB05044FF0004545EA00
:10461000C12145EAC32341EA505143EA525304F110
:104620007F74994204F500344FEAC0204FEAC22259
:1046300008BF904200F09C804FEA13650FF24016CD
:10464000765D4FEA134506FB05F7C7F1807706FB59
:1046500007F74FEAD737A7FB03687642C8F58038DB
:10466000A7FB06CE38BFA8F1010807FB08E64FF00C
:10467000000EA6FB028CE6FB03CEDCF1000CCEF1B3
:10468000004E38BFAEF1010EA6FB0C584FF00007EC
:104690004FF00005E6FB0E87A1FB08C6A0FB07CE86
:1046A00016EB0E0645F10005E1FB076515F1E04E3E
:1046B0007EBFA4F580345FEA46066D4116F180079F
:1046C00045F100054FEA17274FEA066647EA0567F6
:1046D000A6F1DE46B6F1805F4FEA15251FD93846B0
:1046E00024F0010C05EBC471BCF1FE6F01EB0C1161
:1046F00002D8F0BCBDE8008124425CBF01F5801EF9
:104700009EEAC47F02D4F0BCBDE80081244238D4C4
:10471000F0BCA1F1C041BDE8004100F005BA4FEA8C
:10472000D22242EA43524FEAD323A7FB02864FEA42
:10473000D02040EA415007FB03661EEA0E0F4FEA05
:10474000D12105FB026658BFA6EB0056B6EB00561A
:104750004FEA520E4EEAC37E18EB0E0E56EB530E86
:10476000BDD518EB02085E417F1C55F10005B6E788
:104770004FF480154FF000074FF000064FF000088F
:10478000ADE7F0BC4FF0000001F1C04101F0004185
:10479000BDE8008111EA0C1F0CEA131500D00CE0F3
:1047A00013EA0C1F00F025804FF00000F0BC81EAF6
:1047B000030101F00041BDE80081F0BCBDE800410B
:1047C00081EA030100F0B0B9F0BCBDE8004170B56A
:1047D00000F05CF9097EFC3E00F007B881EA0301B5
:1047E0004FF0000001F00041704781EA030100F042
:1047F0009BB9F0BCBDE800414FF000002149704773
:10480000FFFDFBF9F7F5F4F2F0EEEDEBE9E8E6E495
:10481000E3E1E0DEDDDBDAD8D7D5D4D3D1D0CFCD1C
:10482000CCCBCAC8C7C6C5C4C2C1C0BFBEBDBCBB55
:10483000BAB9B8B7B6B5B4B3B2B1B0AFAEADACAB50
:10484000AAA9A8A8A7A6A5A4A3A3A2A1A09F9F9E2A
:104850009D9C9C9B9A9999989797969595949393DC
:10486000929191908F8F8E8E8D8C8C8B8B8A898973
:1048700088888787868585848483838282818180F6
:104880000000FF070000F87F4FEA1153A3F5806393
:10489000D3F11E03A8BFD3F1200C08DB4FF0004278
:1048A00042EAC12252EA505232FA03F070470942FA
:1048B0000BD4102BC4BF0020704703F5787CBCF1EB
:1048C000FF3F05D04FF0FF3070474FF000007047BA
:1048D00070B500F0DBF800BF4992248000207047DB
:1048E000F0E710F0004248BF4042B0FA80F310FAFF
:1048F00003F10AD0C3F11D0303F580634FEA415071
:1049000002EB035202EBD12170474FF000007047D9
:10491000B0FA80F310FA03F10AD0C3F11D0303F5D6
:1049200080634FEA41504FEA035202EBD1217047B6
:104930004FF0000070470000DFF848C170B51CEA76
:10494000111E1EBF1CEA13159EEA0C0F95EA0C0FF0
:1049500000F06F8081EA030423EA4C134EEAD47E10
:1049600021EA4C1141F4801143F48013AE44A1FBC1
:10497000024CA0FB0365AEF17F7E361955EB0C05AA
:10498000A1FB034C4CF10003A0FB021C16EB0C0630
:10499000654153F10003094218BF46F0010613F4C4
:1049A000007F0BD14FEA03314FEA0530340341EA6F
:1049B000155140EA16506FF003020AE04FEAC32196
:1049C0004FEAC520F40241EA555140EA56506FF0D3
:1049D000020202EB2E4201EB025585EACE710AD0AB
:1049E0005FEA440C18BF24F0004450F1000041F18C
:1049F000000120EAD47040F2FE7C624500D270BD16
:104A0000A84214BF4FF080444FF04044002E08BF2E
:104A10000024BEF1806FA8BFA1F1C041BDE8704085
:104A200080F282804FF0000001F1C04101F00041AE
:104A300070479EEA0C0F0CEA131518BF95EA0C0F8D
:104A400006D04FF0000081EA030E0EF0004170BD69
:104A500000F01CF88900013E00F007B800F009B82A
:104A60004FEA430C5FEA5C5C08D081EA030100F086
:104A70005BB84FEA410C5FEA5C5CF6D14FF0000096
:104A8000014970470000FF070000F87F0EF1020E99
:104A90002EF0030E5EF8046B364205D4012A43EB78
:104AA000030515F5001F12D8012841EB010C1CF578
:104AB000001F0CD80ED14FEAD17C15F5001F0CEB6E
:104AC0004C0C0CF1020C08BF4CEBD37C04E04FF013
:104AD000080C01E04FEAD37C0CEB4C0526FA05F6F6
:104AE00006F00706B6F1040C06D20EEB860CBDE804
:104AF00070404CF0010C6047DFE80CF0090B02023B
:104B00004FF000414FF00000A1F5002170BD1946A3
:104B10001046012851EB010418BFD4F5001484BFDE
:104B2000002001F0004170BD0808A0F500114FEA17
:104B3000310170470200FFFF02001027020010271A
:104B40000200FFFF0200E80301020203040506075A
:104B500008090A0B0C0D0E0F1010000000000000D9
:104B6000000001020304060708090000000001021A
:104B70000304000000000000C53600087935000875
:104B8000C1330008113600088D340008753600085E
:104B90006936000809350008F9340008C9350008ED
:104BA00021340008D9330008FD2F0008793B0008A4
:104BB000613C0008213B0008B5390008493A00086B
:104BC000893B0008B1380008593D00084939000800
:104BD000853C0008BD3B00082D330008353800082F
:104BE000493B000899390008553B0008013100088D
:104BF000293C000881390008153D0008ED3B0008FC
:104C0000C93800084F3D0008453D00082133000821
:104C1000E1380008793300080D31000855330008E9
:104C2000B1300008E52F0008A72F00081D3C000840
:104C30005538000847380008A53900083D3B0008F2
:104C4000F13C0008213900086F380008A538000839
:104C5000F9380008713D000819300008303132334E
:104C600034353637383941424344454640305800A0
:104C700030313233343536373839616263646566D2
:104C8000403078000400000800000000000000022E
:104C900000010000103A7474003A7474003A74749D
:104CA00000000000C44C0008000000205C00000070
:104CB00028010008204D00085C0000209C2900000D
:104CC000440100080500024001400000000000000F
:104CD000392C0008752B00080000000000000000BF
:104CE0008D2C0008F92B0008C12B000800000000E3
:104CF00001000000100000000000000000127A0017
:104D00000000000000000000D53600080000000090
:104D10000000000000000000000000000000000093
:04000005080000ED02
:00000001FF
